:020000020000FC
:020000000BC033
:02000C0038C0FA
:1000160046C00DE40DBF04E00EBF09E00EBD00E1D1
:1000260009BF10E000EA1BBD0ABD10E00FEC10BDD1
:1000360009B908E90AB90EE800BD0FEF07BBCEE41F
:10004600D4E006E90993099309930993099309935F
:1000560009930993099309930993099309930993BA
:1000660009930993CEE4D4E078940881201710F41C
:10007600C198FBCFC19AF9CF4FB7F8942395283C86
:1000860060F03395532F551F551F58BBC395222734
:10009600303118F03327CEE4D4E04FBF18954FB770
:1000A600F8945F9BFCCF5CB15F3F19F4AEE4B4E01B
:0C00B60003C0CF3509F05D934FBF1895D3
:00000001FF
